:030000000219FDE5
:03000B000200AA46
:03002B0002018748
:03005B0002033667
:0300730002032362
:1000800002030406080C10182030406080040608A3
:100090000C10182030406080A0C00003070F1F0D17
:1000A0000D0403060D0503030202C2AF306308C24C
:1000B0006385798AD2AF32C0D0C0E0206221E525C5
:1000C0006016E473E525F4C3334009758A00D263F2
:1000D000F57901D6F58AD262D0E0D0D0D2AF32C362
:1000E000E526334009758A00D263F57901F0F58A77
:1000F000C262E526F4602F30682520720DD0E0D072
:10010000D0C292C296C294D2AF32C292C296C29468
:10011000206F0C206609740ED5E0FDE57B4290D07F
:10012000E0D0D0D2AF32758A00D263757900C28D2B
:10013000D262211F01C4306805206602D29201C438
:10014000306805206602D29401C43068052066023A
:10015000D29601C4C29330680A2066077410D5E0B5
:10016000FDD29201C4C29530680A2066077410D58A
:10017000E0FDD29401C4C29730680A20660774106B
:10018000D5E0FDD29601C4C2AFC2AD53E6EFC0D0F8
:10019000C0E0D2D3D2AFE57A6009E5776005757724
:1001A00000412C757701C2CEE52A600720744915FD
:1001B0002A21F87800790020742EE580307E01F441
:1001C00030E50278FF53DACF207E0343DA20307E19
:1001D0000343DA10C2D8C271E580307E01F430E505
:1001E0000279FFC3E89970CB306103752A4020740F
:1001F00003752A40885CD27020740DE52B600415CD
:100200002B410843DA01C2D8207002411BA85C20B0
:100210006102C270207402411988227882B60403F8
:10022000852224C3E52594404002D26420CF0AD021
:10023000E0D0D043E610D2AD32C2CF053AE57A60C5
:1002400009E578600575780061197578017802E52F
:100250002A6005307402152AC3E55C9401400575D7
:100260005F004175756000756900E55F2401F55F09
:100270005003755FFF7982B7020D306E1DC3E52212
:1002800094324016854C227982B7030E306E0BC330
:10029000E52294324004798E8722C3E523952260BB
:1002A000084004152341A90523D8CA0569E56970EA
:1002B000021569D56A63756A017805C3E569956BAE
:1002C0004057C3E569956C50087801756A030202CE
:1002D000DDC3E569956D50057801756A01C3E56276
:1002E0009524401E7982B70402610E206E14852485
:1002F00062E569046003856B69756A0175233C02D8
:100300000319E5622850057562FF610EF562E5622A
:100310000470067560FF7569FFD0E0D0D043E61029
:10032000D2AD32C2AF53E67F7592FA7593FFC260C9
:10033000759104D2AF32C2AF53E6EFC2ADC0D0C0A8
:10034000E0C0F0D2D3D2AFA8FBA9FCE57A6007C326
:10035000E913F9E813F8C2D830710261A853DACF73
:10036000207E0343DA10307E0343DA20D271E58029
:10037000307E01F420E502617F88278928A18D5312
:10038000DACF207E0343DA20307E0343DA10C2D86E
:10039000C271307402A1797800E580307E01F430BA
:1003A000E502A179885CA16153DACF207E0343DAAC
:1003B00020307E0343DA10C271206102818153DA5A
:1003C000CF207E0343DA10307E0343DA20C2D8D236
:1003D0007188578958C3E89555F8E99556F97B0017
:1003E0007E087A00C3E8948CE994005005755B00A0
:1003F0008173882178A2E6A8216055C3E894C8E9F2
:1004000094005008E4D2E4FB7A0A814EC3E8946871
:10041000E994015008E4D2E3FB7A0F814EC3E894DB
:10042000D0E994025008E4D2E2FB7A1E814EC3E880
:1004300094A0E994055008E4D2E1FB7A3C814EC3D4
:10044000E89498E994085008E4D2E0FB7A787E00BA
:10045000C3E89559FCE9955AFD30E70AECF424010C
:10046000FCEDF43400FD755B00C3EC9AED9E500387
:0F047000755B018859895A85575585585678020A
:10047F00A161C3E89527F8E99528F9307C02A145D9
:10048F00307B02A145307A02A13E20750281A4E99A
:10049F00FDE8FC81C3E9C313F9E813F8307902A131
:1004AF003EE9C313F9E813F8307802A13EE9C3130C
:1004BF00FDE813FC20612CC3EC941CED9402400268
:1004CF0081DAED701EC3EC94C850180529E5297028
:1004DF00021529C3E529940A5002A179755C00D24F
:1004EF0070A179E529600215297400207F037896A1
:1004FF00E624FAFEE43400FFC3EC9EFCED9FFD50B2
:10050F000678007900A145C3EC94FFED94004006F6
:10051F0078FF7900A145EC8572F0A4C5F0A2F733FE
:10052F00F87900400302056178FF7900020561E95F
:10053F00C313F9E813F8307C0EE9600278FFC3E8C3
:10054F001338F8E43400F9C3E894FFE9940040024B
:10055F0078FF885CD270206102A179741FF4552F47
:10056F004BF52FC274EB7002D274752A40307403AE
:10057F00752A0A306102A18D20740353DAFE2074AC
:10058F0003752B20D0F0D0E0D0D0D2AD43E610329F
:10059F0079010205BD79030205BD790A0205BD790E
:1005AF001E0205BD79640205BD79C80205BD781725
:1005BF00E4D5E0FDD8FAD9F6227A147B780205E467
:1005CF007A107B8C0205E47A0D7BB40205E47A0B7A
:1005DF007BC80205E47902E4C295D5E0FDD294D53B
:1005EF00E0FDC294D5E0FDD295D5E0FDE920E00213
:1005FF00D29230E002D296E573D5E0FDE920E00219
:10060F00C29230E002C2967496D5E0FDD9C9EAF8DD
:10061F00D5E0FDD8FBDBBEC29522C37C007D007503
:10062F00F00005F0EA33FAEB33FB50F6EB13FBEA7D
:10063F0013FAC3E9FFE8FEE89AF8E99BF95004EFD3
:10064F00F9EEF8B3EC33FCED33FDD5F0DFEDF9EC5B
:10065F00F822E889F08A20D2D4F8A9F07B0030F78D
:10066F000B7BFFF42401F8E9F43400F9E88520F05E
:10067F00A4ADF0F8E98520F0A4AFF0FEED2EF974EB
:10068F00003FFA7C04C3EA13FAE913F9E813F8DC24
:10069F00F48BF030F70AE8F42401F8E9F43400F9A8
:1006AF00E889F0C2D4F8A9F0227882B604030207D1
:1006BF0057C3E55C9419401EE52D54067018206E43
:1006CF003678057994E7146007780A146002781277
:1006DF00C3E54198401F306E098564627569FF75E7
:1006EF006A01852224E4F544F545F546F547F548BA
:1006FF00C26E020757D26E7994E7147013E523F494
:10070F003333F913F8E9540104F9E854FE02074BA7
:10071F00E714147014E523F4333333F913F8E95461
:10072F000304F9E854FC020753E523F4333333335E
:10073F00F913F8E954070404F9E854F8C39440F89E
:10074F00E99400F98844894522C3E54113F9E5404E
:10075F0013F8C3E54498F8E54599F9500CC3E894AC
:10076F0080E994FF401602078FC3E8947FE9940055
:10077F00500302078F787F790002078F788079FF07
:10078F008849894A22E5492546F8E54A3547F985DA
:10079F004A20E4300701F43548FA30E709C3EA94F8
:1007AF00F040150207CDC3EA940F50030207CD782E
:1007BF00FF79FF7A0F0207CD780079007AF0C3E551
:1007CF00249561500AC374019524500B0207EBE581
:1007DF004A20E70E0207EBE54A30E70688468947CD
:1007EF008A482278A5E6FAC3E54933F8E54A33F992
:1007FF00120661E930E70BC3E89480E994FF4013D8
:10080F000126C3E8947FE9940050020126787F798E
:10081F00000126788079FFE820E715C3E52398F8D3
:10082F004009C3E89401400302084D780102084DC6
:10083F00E8F424012523F8400302084D78FF884B84
:10084F002278A6E6FAA847A948120661E930E70C14
:10085F00C3E89401E994FF4016020882C3E894FFAD
:0F086F00E99400500302088278FF7900020882A2
:10087E00780179FFE920E715C3E54B98F84009C3E5
:10088E00E8940140030208A978010208A9E8F424BB
:10089E0001254BF840030208A978FF88242278FF2F
:1008AE00C26420693D206A12D264C3E541940A40B5
:1008BE0009C3E52594405002C26479A1E76023E59F
:1008CE0041601F74FF8541F0848539F0306A0375ED
:1008DE00F005A4F8C5F0600278FFC3E895645002F5
:1008EE00A864886322C3E54094C8E5419400E5639B
:1008FE005003142104046002F563227883E6F52088
:10090E00120FA475E89012059F75E890E5E820ECAB
:10091E00FBA8BDA9BE12104A756E00756F00C37498
:10092E000013FD7400606613FC74002CFC74003D13
:10093E00FDECFAEDFBC3E89AE99B4014E56E24004A
:10094E00F56EE56F3400F56FEA2CFAEB3DFB80E5B2
:10095E00AE6EAF6FC3E56F13F9E56E13F8C3E9130F
:10096E00F9E813F87A03C3E913F9E813F8DAF7AAEA
:10097E00201A7009756E00756F0002099B1AEA60E5
:10098E0008EE28FEEF39FFDAF88E6E8F6F2275E8CB
:10099E0090227883E6FFE5E820ECF7A8BDA9BE0516
:1009AE0070C3E57094084052757000E9FA79A0E7BB
:1009BE006044EA7007E571601B0209D6C3E89571C1
:1009CE006010E5715006600C140209E20460F90231
:1009DE0009E2E571F571C39472401B7561C0C39451
:1009EE00044013756180C39404400B756140C39439
:1009FE0004400375610075BB0822EFC39401601FAC
:100A0E007400601BC3E894FFE994035012C3E89589
:100A1E006EE9956F5009E561600C1561020A34E5C7
:100A2E0061F460020561A861C3E524985002A82410
:100A3E00C3E89562400AA862E562F46003856261CC
:100A4E0088258826E570B4070375BB1022743279A9
:100A5E00A787F0A4C5F0A2F733F8C3E8956140026A
:100A6E00A8618822882488258826886422754000FB
:100A7E007541F022C2AF75C820A8CCA9CDAA3A30D4
:100A8E00CF010A75C824D2AFC3EA13FAE913F9E805
:100A9E0013F8AB3BAC3C883B893CC3E89BF8E99C24
:100AAE0020690A547FF9306702619C41F9AD3D8A95
:100ABE003DF9EA9D547FFA600478FF79FFAE3EAFB0
:100ACE003F8B3E8C3FA83BA93CC3E89EF8E99FF9BB
:100ADE00C3E54113FBE54013FAE82AF540E93BF57F
:100AEE004150067540FF7541FF6143AA40AB41ACD2
:100AFE0040AD417E047F02C3EB940440021E1FC32F
:100B0E00EB940840021E1FC3ED13FDEC13FCDEF741
:100B1E00C3EA9CFAEB9DFBEF6009C3E913F9E813F6
:100B2E00F8DFF7EA28FAEB39FB8A408B4150067B57
:100B3E00FF8B408B41C3EB94025002D267306904A5
:100B4E007F03616E7892E6FFC3E537948240110F02
:100B5E00C3E53794A040010FC3EF940640027F0512
:100B6E007E02E541C4540FF9E541C454F0F8E54066
:100B7E00C4540F28F8C3E89EFAE99400FB4009C359
:100B8E00EA9402EB940050047A02E4FB61E8AA4076
:100B9E00AB41EBC4FEEAC4540F4EFCC3EA9CFAEB25
:100BAE009400FBC3E813C313F8EA28FAEB3400FBF6
:100BBE008A408B41C3EB94024002C2677802EBC4B9
:100BCE00FE7B00EAC4540F4EFAC3EA98FA4005C3FE
:100BDE00940250027A027892E6FF30600261E88554
:100BEE005192855293D26043E680C3E49AF8E49B17
:100BFE00F9C3E833F8E933F9306702817BE8FAE9A3
:100C0E00FBD3E913FDE813FC88518952C3EF94031B
:100C1E006038EF20E00DE82CF8E93DF9ECFAEDFB39
:100C2E00020C44E828F8E939F9C3E82402F8E9345B
:100C3E0000F97AFE7BFFC3EF9403400E8A538B5468
:100C4E00884D894E8C4F8D5081AF885389548A4D73
:100C5E008B4E8C4F8D503069127553F07554FF7555
:0F0C6E004FF07550FF7551F07552FF81AFE8FAE6
:100C7D00D3E813FC8851C3EF94036020EF20E00705
:100C8D00E82CF8ECFA819BE8282402F87AFEC3EFF1
:100C9D00940340088A53884D8C4F81AF88538A4DF9
:100CAD008C4FE568C3335002646BF5683060028188
:100CBD00B9753402D26043E680E52D5406602DA847
:100CCD0040A941C3E913F9E813F8306904E9244058
:100CDD00F9C2AF53E67F759100C3E498F594E4999A
:100CED00F595759104D26043E680D2AF22D2657539
:100CFD004300752000306C03752040020D19D2653C
:100D0D00754300752040306C037520007801790122
:100D1D00206720E52D54066002C2657914E541C3B4
:100D2D0013700104F8C394144002781430690478E8
:100D3D001B791BC3E833F8C3E933F9206010E54391
:100D4D00600C306903D53404D26DA1D191C1054336
:100D5D00E59BF45440B52002A1BB30690908C3E8F6
:100D6D0099400118A14820650A08C3E8994002A1DD
:100D7D0019A148C265C2AF53E67F75910030671265
:100D8D007594007595FC759104D26043E680D2AFE1
:100D9D00A119AE40AF41C3EE33FEEF33FF50047ED9
:100DAD00FF7FFFC3E49EF594E49FF595A193C3E502
:100DBD003394015002A119306502A119D802A1CFB7
:100DCD00A148C26DC2AF53E67F75910085539485DE
:100DDD005495759104854D92854E93D26043E6806E
:100DED00D2AFE52D54066008206A020533020E0DC0
:100DFD00306D0D206C0A206507158115810216A531
:100E0D002278003064053065027801E53775F0070A
:100E1D00A4F9E5F028F5F0E9A2F013A2F113A2F27E
:100E2D0013F537C394785003753778C3E537953884
:100E3D004008D266C292C296C294306002C1478504
:100E4D004F92855093D26043E68022207D16C2AF2B
:100E5D00754202C295D293306202D296D2AF759F7F
:100E6D0040021047C2AF754202C295D2973062025E
:100E7D00D292D2AF759F40021047307243207D2031
:100E8D00C2AF754203900165757B20C296C2973043
:100E9D006204D294C1A5D295D2AF759F410210477D
:100EAD00C2AF754203900165757B20C292C293302B
:100EBD006204D294C1C5D295D2AF759F430210473B
:100ECD00207D17C2AF754203900140C29630620279
:100EDD00D294D2AF759F41021047C2AF75420390B5
:100EED000140C292306202D294D2AF759F4302107C
:100EFD0047207D16C2AF754204C293D2973062026D
:100F0D00D294D2AF759F43021047C2AF754204C24F
:100F1D0097D293306202D294D2AF759F410210479F
:100F2D00307243207D20C2AF754205900154757B10
:100F3D0008C294C295306204D292E14BD293D2AFE3
:100F4D00759F40021047C2AF754205900176757BC3
:100F5D0080C294C295306204D296E16BD297D2AF23
:100F6D00759F40021047207D17C2AF754205900155
:100F7D0036C294306202D292D2AF759F40021047B2
:100F8D00C2AF75420590014AC2943062EBD296D23F
:100F9D00AF759F40021047207D16C2AF754206C245
:100FAD0097D295306202D292D2AF759F410210470F
:100FBD00C2AF754206C293D295306202D296D2AFBD
:100FCD00759F43021047307243207D20C2AF75429A
:100FDD0001900176757B80C292C293306204D296E5
:100FED00E1F1D297D2AF759F43021047C2AF754260
:100FFD0001900154757B08C296C297306204D2925B
:10100D000111D293D2AF759F41021047207D17C2B7
:10101D00AF75420190014AC292306202D296D2AFB0
:10102D00759F43021047C2AF754201900136C296BB
:10103D00306202D292D2AF759F41C26622900134C6
:10104D00757B00C292C296C294C293C297C295C2DA
:10105D0062227880760708760708760108760408FC
:0F106D0076FF0876FF08760A08760208760108F3
:10107C007601788C76010876000876B40876FF083D
:10108C0076FF0876FF0876030876FF087601087667
:10109C00FF0876250876D00876780876C808760496
:1010AC000876FF08760108760008767A08760A0832
:1010BC0076010876010876000876FF08760022781B
:1010CC0087E6FFC272BF0302D2727888C27DE63017
:1010DC00E102D27DC27E7889E630E102D27EC3EF96
:1010EC0094026008758E01D2730210FD758E00C2D9
:1010FC0073227880E6149000809378A5F67881E6C8
:10110C00149000809378A6F67886E61490008D9360
:10111C0078A7F6789FE6F8700108C3E894114002AE
:10112C007811E82828F56B256B256B28F56C256B59
:10113C002828F56D7886E6F539C394025003753985
:10114C0002789CE67538FFB402037538A0B403032B
:10115C0075388278A3E61490009A93F566114A22AA
:10116C00227896E6FA7897E6FB7888E6B40305C30E
:10117C00EB940EFB307F047A007BFFC3EB9AFCC32D
:10118C00948250027C827572000572EC8572F0A418
:10119C00C3E5F0947D40F222D27F316D1205AE7A18
:1011AC00007B007C101205A4E55C2AFA74003BFB62
:1011BC00DCF37C04C3EB13FBEA13FADCF7FEC27F0F
:1011CC00316D22E5EF20E6037520000520903FFFEE
:1011DC00E520146006901FFF1460009304600375F3
:1011EC00EF1253D9BF7581C043FF8012059F75EF75
:1011FC000243B203E5B3240220E70DF521E5E32019
:10120C00E0068521B343E301114A7580FF75A40004
:10121C0075F13075D4DF75900375A5FC75F2FC750E
:10122C00D50175A60175E241C292C296C29412050F
:10123C00B3D293D297D29512059FC293C297C295FF
:10124C00114AE4F8F6D8FD756801115F121703789E
:10125C00988673753001C2AF1205B81205C8120515
:10126C00AE1205CF1205AE1205D61205AE12182518
:10127C001205B81205B81205B3C2AF78FA79FA3074
:10128C008507D9FBD8F7021C0011CB11FE316C314C
:10129C006D78988673114A75A90075B680757A00B9
:1012AC0075881075890275C82475910475D84075B8
:1012BC00A82275B80275E690759B80759D0075D156
:1012CC000E75BCC075BB0875BA1175E88012059F08
:1012DC00D2AF12090975360053DACF207E0343DAF8
:1012EC0020307E0343DA1043DA01C2D8C2711205F2
:1012FC00B8D2617B037A0CE55B70077A0CDB0302D6
:10130C0012851205AE207003021285C270E55CC313
:10131C00940240E1E52F541F855E5DF55EB55DD509
:10132C00DAD5C26153DACF207E0343DA20307E0354
:10133C0043DA10C2D8C27178A2E67008D274E52FD5
:10134C0054E0F52FC2757529001205B3307409C32A
:10135C00E529940A4002D2751205A4780230740271
:10136C007800C3E55C9840F0C2AF1205C81205C8FE
:10137C001205C8D2AF1205B8754C001205A4788CB2
:10138C00E6C39401500302145DE530C3940150038D
:10139C0002145D207435C3E55C94FF500302145DA8
:1013AC00C2AF1205DDD2AF1205B3C3E55C94015098
:1013BC00EFC2AF1205C81205A91205C8D2AF1205AB
:1013CC00B3C3E55C94FF40E90218AA7F05D27F31D4
:1013DC006D1205B3C2AFC27F316DAE5CC3E55C94D8
:1013EC007FD2AF407612059FC2AF1205DDD2AFDFC0
:1013FC00DC31A4C3EE94057897F61205B8121744A5
:10140C0012182D7F0AD27F316D1205B3C2AFC27F85
:10141C00316DAE5CC3E55C947FD2AF50E612059F94
:10142C00C2AF1205C81205A91205C8D2AFDFD6315A
:10143C00A4EE24037896F61205B812174412185C21
:10144C001205B3316DC3E55C94FF5002619F021825
:10145C00AAC3E55C954C4003855C4C1205B378013E
:0E146C007988E7B403027805C3E55C98400276
:10147A006187C2AF1205DD1205DD1205DDD2AF129A
:10148A0005B8753000E4F531F5320531E531F4700F
:10149A003E0532789AE67819146012783214600D93
:1014AA00787D14600878FA146003753200C3E53257
:1014BA0098401C114A12059F153275310078998699
:1014CA0073C2AF1205DDD2AF789886731205B312D4
:1014DA0005A9E52A70053074024185780120740255
:1014EA007806C3E55C9840A21205B3E52A700302A8
:1014FA001285C2AF114AE4F522F523F524F525F544
:10150A0026F567D2AF7885E6C333F565E4F544F589
:10151A0045F546F547F548F570F52CF52DF537757F
:10152A00700875BB1012059F12099CE5E820ECFBB8
:10153A00A8BDA9BEE97001F888711209A0757008E2
:10154A0075BB1011CBC2AF7561FF120A5B852261B0
:10155A00852262852263D2AF752201752401752521
:10156A0001752601856069756A0175B69075A903CA
:10157A00757A017888E6B40307C27D307602D27D97
:10158A00D268D269753300120FA4120FD3120A7BE4
:10159A00120A82120A7B120A82120A7B120D0B129B
:1015AA0006B8120E0E120E58120A82120CFA306E79
:1015BA00031207582067031208AC3067031208F3B6
:1015CA00120E0E120E87120A82120D0B306E0312C1
:1015DA000794120E0E120EFE120A82120CFA306EC6
:1015EA00031207F2120E0E120F2D120A82120D0B9F
:1015FA00306E03120850120E0E120FA4120A821233
:10160A00099C120CFA120E0E120FD31209A0120A1A
:10161A008230692C856461856462856069756A01B6
:10162A0079187A0CC3E533994009C269D26A8A35B6
:10163A0002164AC3E55C940140030215A60216ADE0
:10164A00306A1D206C1AE535147006C26AD26BA185
:10165A00A6F535C3E55C940140030215A60216AD52
:10166A00753600C3E55F9401400985646285606947
:10167A00756A0178FA79A4E760027803C3E55F988E
:10168A005021307404E52A601A78F0306C058564BC
:10169A00617820C3E541985002A1A60536E55C6051
:1016AA0002C1B0753600C2AF114A7887E6FE7602EB
:1016BA0011CB7887EEF6E4F522F523F524F525F526
:1016CA0026F565752C00752D0075A90075B680750F
:1016DA007A00D2AF1205B3114A78A4E66006D29313
:1016EA00D295D297307406E52A70024185788DE644
:1016FA00C3940140026164818F901A0D78201217F9
:10170A0086E520B4A50CA3121786E520B45A030275
:10171A001724115F121744021743901A0378807B2B
:10172A000A121786A308DBF9901A0F788C7B191214
:10173A001786A308DBF9901A2822C2AF1217C5121E
:10174A00179F901A00740E12178BA3740612178B28
:10175A00A3741512178B901A0378807B0A12178AC2
:10176A00A308DBF9901A0F788C7B1912178AA30841
:10177A00DBF91217D81217B6901A2822E493F62228
:10178A00E6438F01538FFD75EF0275B7A575B7F163
:10179A00F0538FFE22438F02438F0175EF0275B714
:1017AA00A575B7F1901A0DF0538FFC22901A0D749B
:1017BA00A5F18B901A0E745AF18B227A3079D0786F
:1017CA0020901A40F186E520F709A3DAF7227A3049
:1017DA0079D0901A40E7F18B09A3DAF922AB74A801
:1017EA0075BB01027980BB02027981BB030279824F
:1017FA00BB04027994BB05027983BB06027986BBD6
:10180A0007027992BB08027987BB0902799CBB0A55
:10181A00027988BB0B027989E8F7227C051205B8A0
:10182A00DCFB22C2AF1205C81205CF1205D612057B
:10183A00DD1205A91205C81205CF1205D61205DD5B
:10184A001205A91205C81205CF1205D61205DDD256
:10185A00AF22C2AF1205DD1205D61205CF1205C896
:0F186A001205A91205DD1205D61205CF1205C809
:101879001205A91205DD1205D61205CF1205C8D227
:10188900AF22AE74AF75C2AF1205C81205C81205F2
:10189900C81205A9DEF21205DD1205A9DFF8D2AFDB
:1018A90022112D11251125757401757501757600A3
:1018B900118B7C05AD5C1205B8C3ED955C70F5C361
:1018C900E55C9401400AC3E55C94FF40340218E8E2
:1018D9001217E7121744112DC2AF75EF121125DC4B
:1018E900D30576C3E5769403500280C411250575A6
:1018F900E5741490009F93F808C3E5759850028029
:10190900AC112511250574C3E574940C5002809A15
:0D19190012105F121744C2AF75EF121125B6
:0319FD000211CF05
:101A00000E061507070104FFFF0A020101A55A018E
:101A100000B4FFFFFF03FF01FF25D078C804FF01DA
:091A200000FF0A010100FF00FFB4
:101A400023475F556C74726132304123202020207F
:101A500023424C48454C492346333930232020202B
:101A60002020202020202020202020202020202076
:101C0000C2AFC2D353D9BF7581C043B20343FF8073
:101C1000752438752503B1C975EF0275E24043F1AB
:101C20002053A4DF75D4FFD2857DFA780379E67C52
:101C300010752200752300901DD67B0675249875BB
:101C400025013085028142208508D8FBD9F9DCF7CF
:101C500081B4308508D8FBD9F9DCF781B4B189E4C7
:101C600093A3C39A6004DDC381B4DBDBB17B600264
:101C7000812B7B08E493FAA3B15CDBF87A30B15C8A
:101C8000752200752300B17BEAFCEBFDC3ED94FEE9
:101C9000400EB17B8A278B28ED30E0048A828B834B
:101CA000B17B7AC270D8C3ED94FE601350CEBD00F4
:101CB00025EC60097520007521FF0200008100A855
:101CC00027A9280809D804D90281D3B17FEA89AAB3
:101CD000F281C50D81A0C3ED94035049EDA2E092BD
:101CE000007AC5C3E5829400E583941C50902000DF
:101CF00010438F02438F0175B7A575B7F1F030001F
:101D00001FA827A9280809438F01538FFDD804D99C
:101D100002A12089AAE275B7A575B7F1F0A3A10DBC
:101D2000538FFC817C7AC1BD030CE493A3FAB140CC
:101D3000DCF8B138817C817EAA22AB23B15CEBFA5E
:101D4000EA6222752608C3E52313F523E52213F57D
:101D50002250066323A0632201D526EAB1C9B1C986
:101D600075260AEAF4200102D285300102C285B14B
:101D7000C9C3134002C201D526EB22B17FEAFB2082
:101D80008502A17F308502A184752608AE24AF2587
:101D9000C3EF13FFEE13FEB1CDB1C9C3EA13308513
:101DA000024480FA30E703632201C3E52313F523DD
:101DB000E52213F52250066323A0632201D526D91C
:101DC000E52265236523F52222AE24AF250E0FDE22
:101DD000FEDFFCD20122424C48656C693437316326
:041DE000F390060175
:00000001FF
